:0800000040C096C0E4C0FCCF33
:10000800FBCFFACF33C1F8CFF7CF18C1F5CFF4CF74
:10001800F3CFF2CFF1CFF0CFEFCFEECFEDCFD804C3
:10002800F6041405320550056E058C05AA05C805A9
:10003800E6050406220640065E067C069A06B80611
:10004800D606F406120730074E076C076C076C07D4
:100058006C076C076C076C076C076C076C07010072
:100068000000000000003B003B303B303B303B30A1
:100078003B0001009B0166000000F894EE27ECBBF2
:10008800F1E0FBBFEBBFE5BFF8E1F1BDE1BD8DE0FD
:10009800A2E0BB27ED938A95E9F780E094E0A0E61B
:1000A800ED930197E9F7EAE7F0E0859195910097DC
:1000B80061F0A591B59105901590BF01F0010590EB
:1000C8000D920197E1F7FB01F0CFEFE5EDBFE4E01A
:1000D800EEBFC0E6D1E001C3AF93AFB7AF93BF9314
:1000E800A8E0B881AA23C9F0AA958894BB1F18F084
:1000F800C09804D0F7CFC09A01D0F4CF0000000018
:100108000000C19A0000000000000000000000008C
:10011800C1980000000000000895C098BF91AF91F9
:10012800AFBFAF91219608950A921A92FA926A93F4
:100138007A938A939A93AA93BA93EA93FA93EFB726
:10014800EA932197E0911C02E150F9D3E0911B0258
:10015800F9D3E456FE4F1080E0911C02A1E022D5AD
:10016800E121E883E03011F4C09801C0C09AE09121
:100178001C02E03031F4E0911B02EF5FE5D3E1505F
:10018800E6D3E7D3A0911B02B0E0EA17FB0760F4BF
:10019800E0E0DAD3DCD3EBB7EF7BEBBFC29A000029
:1001A800C298DCD3C29AE0D32196E991EFBFF991C6
:1001B800E991B991A9919991899179916991F99068
:1001C800199009901895689422F8AF93AFB7AF9338
:1001D800BF937894A2B7F894B0918601A093860152
:1001E800AB1BA0938A01A0918301B0918701A093D2
:1001F8008701AB0BA0938B01A0918401B09188017A
:10020800A0938801AB0BA0938C01A0918501B091BC
:100218008901A0938901AB0BA0938D01A09197014F
:10022800A395A093970129F4B0919801B395B09341
:100238009801BF91AF91AFBFAF911895AF93AFB78A
:10024800AF93A0918301A395A093830159F4A09142
:100258008401A395A093840129F4A0918501A39515
:10026800A0938501AF91AFBFAF9118956A937A9328
:100278008A939A93AA93BA93EA93FA93EFB7EA9375
:10028800E0911F02F09120023196E0931F02F09353
:100298002002E0E022FCE1E0E13090F0E0918A0108
:1002A800F0918B0160918C0170918D0163D368D4BA
:1002B8006AD3E0919201EF5FE0939201E89422F80B
:1002C800A0911F02B09120025497C8F0E0919701C5
:1002D800F0919801E0939901F0939A01E0E0E0939E
:1002E8009701E0939801E0E0E0931F02E093200279
:1002F800689420F8E0911D02EF5FE0931D02E991F8
:10030800EFBFF991E991B991A99199918991799161
:1003180069911895E881E06CE7B98BE18A95F1F766
:10032800369A349BFECF349AE4B1F5B121960895FC
:10033800229732D3AFD4EF2FF0E0E983FE01319654
:10034800DF01EC91E06AEC9327D3E491E883C2984B
:10035800EEE82CD3E0E62AD3C29A0000C298E981DD
:1003680025D3E88123D3C29A0000C298E0EB1ED3BC
:10037800C29A0000C298E8EC19D3EFE817D3C29AE2
:100388000000C298E2EC12D3E0E210D3C29A000057
:10039800C298E2ED0BD3E0E409D3C29A0000C298F8
:1003A800DDD2C29A22960895689423F8D0D2E0E06C
:1003B800CBD2E0E4EABFC298E0ECF8D2E8E3F6D2A8
:1003C800C29A0000C298E6ECF1D2EBB7E064EBBF4A
:1003D8000895E0E0EDD2F1D2E1E0EAD2F7D2E6E02A
:1003E800E7D2FDD2E2E0E4D203D3E3E0E1D209D3DD
:1003F80011D3139750F4E0E0E0939301E093940154
:10040800E0939501E09396012FC004D3AE35E1E067
:10041800BE0770F4E091920102D3FBD3B4D2E0910D
:100428009B01FDD2D1D3A0EEB0E782E790E01AC0DD
:10043800E0919901F0919A01F7D2F9D2A091930134
:10044800B09194018091950190919601ECE3F0E0D0
:1004580060E070E0B9D3DF01CB01E0919B01FF2799
:1004680066277727D6D3E3D2E0E0E0939901E093BB
:100478009A01E0E0E0938E01E0938F01E093900110
:10048800E0939101E0E0E0939201DAD2A091620159
:10049800B09163018091640190916501D6D28DD2AB
:1004A800CFD2A0916601B0916701809168019091C7
:1004B8006901CBD28BD2E0918001F0918101A091AA
:1004C8006A01B0916B0180916C0190916D01BDD270
:1004D80086D2C5D2CDD251F4E0E0E0936E01E0932C
:1004E8006F01E0937001E093710112C0F894E091FC
:1004F8007601F0917701B3D2C3D2C4D2DF01CB0128
:10050800E0917A01F0917B01BBD2A8D371D27894A3
:10051800C0D2AED251F4E0E0E0937201E0937301EF
:10052800E0937401E093750112C0F894E0917801AA
:10053800F0917901AED2A4D2A5D2DF01CB01E0912E
:100548007C01F0917D019CD289D35BD27894089587
:10055800259785E0A0E0B0E0E8E6F0E0C2D3F9D165
:10056800E983E5E0E883E981A881AE1748F49AD2E7
:10057800E081AA81EA27EA83E881EF5FE883F3CF85
:10058800EA81EB83EA81E07FEA83E295EF70EA8310
:10059800AA81AA3010F0E95C02C0EA81E063EA832C
:1005A80086D2EF70EC93AB81AA3020F0EB81E95C46
:1005B800EB8303C07CD2E063EC93E0E0EC837CD275
:1005C800FE0134967ED2B4D2259608952B97EAEA96
:1005D800E0939C01E0939D01E0939E01EDE2E0939E
:1005E8009F01E4EDE093A001E4E2E093A101E3E3DD
:1005F800E093A201EBE3E093A301E1E3E093A4011C
:10060800EBE3E093A501E0E0E093A6015DD259D2C7
:1006180060D229D151D25DD25FD260D2E09162011D
:10062800F091630160916401709165015BD251D2D0
:1006380053D254D2E0916601F0916701609168014C
:10064800709169014FD245D247D248D2E0916A01F0
:10065800F0916B0160916C0170916D0143D239D2B8
:100668003BD2E0E7F0E02DD272D2E0916E01F0913A
:100678006F01609170017091710134D22AD22CD22D
:100688002DD2E0917201F091730160917401709123
:10069800750128D21ED220D221D2E0919301F09187
:1006A800940160919501709196011CD212D214D2D6
:1006B80015D24EDF4ED1E883F5D1ADE0A083E881B5
:1006C80041D1E356FE4FAAE0A083E8813BD1E25630
:1006D800FE4FA0E0A0832B960895E0E0E09382010E
:1006E800E0938301E0938401E0938501E0E0E093E7
:1006F8008601E0938701E0938801E0938901ECE3A8
:10070800E8BBE7E0E7BBE0E3E5BBE0E0E4BBE0EE45
:10071800E2BBE2E0E1BBE3E0E3BFE0E0E2BFEFBD64
:10072800EAE0EEBDE0E0EDBDECBDE7BDE6BDE3EC23
:10073800EBBDEFE4EABDE0E0E9BDE8BDE2BDE5BD43
:10074800E4BDE3BDEBB7E068EBBFEAE0E5BFE0EC92
:10075800EABFE1E1E9BFE0E8E8B9E0E0E0BFE0ECEA
:10076800E7B9E5E8E6B9A8E0B0E09DD2E0937E01FC
:10077800F0937F01AAE0B0E096D2E0938001F09375
:100788008101A0E0B0E08FD2E0937601F093770189
:10079800A2E0B0E088D2E0937801F0937901A4E078
:1007A800B0E081D2E0937A01F0937B01A6E0B0E05B
:1007B8007AD2E0937C01F0937D01E3B3E295E37094
:1007C800EF5FE0939B01E6B3E695E695E695E77063
:1007D800E0931E02E0B3E695E695B4D0E070F271BE
:1007E800A0911E02EA2BE0931E02A2DD789420FE5F
:1007F80002C023FE01C00CC0ECDDE8DEE89420F85E
:1008080063D13196E0936001F0936101689421F817
:10081800E0E023FCE1E0A0E0D2D10E2EE0E021FCF4
:10082800E1E0A1E0CCD1E02119F0BEDDE89421F8A7
:10083800A0911D02A330A8F0F894E0E085D087D0FD
:10084800EBB7EF7BEBBFEAB7E064EABFC29A000000
:10085800C29884D0C29A88D06BDDE89420F821F839
:100868007894C5CFFFCFA991B991E991F9913096C4
:100878002AF4E095F09531966DE26D93E89480E165
:1008880097E20DD088EE93E00AD084E6992707D046
:100898008AE005D06E2F10D066276C9308956627DE
:1008A800E817F90720F06395E81BF90BC9F76623E9
:1008B80011F416F008956894605D6D930895249777
:1008C8000AD2E0E0FAEC6AE97BE312D100E015D144
:1008D800FED14CF4E885F9856A857B855BD112D118
:1008E80016D1EDE2EC931AD194D11E2F103059F4A1
:1008F800003049F418D1A130E0E0BE07E0E08E07EF
:10090800E0E09E0729F403D1E12FE05DEC9301E0DC
:1009180005D1A9D1F7D007D1EAE0F0E060E070E0B6
:1009280078D1E6D0EA81FB816C817D81CCD1D9F682
:10093800AE81BF81E0E0EC93D1D12C960895E0938D
:100948001C020895F0E00895E0931B020895E8E082
:10095800F6CFECE9F1E0FA93EA9308C1E0ECEA9308
:10096800BBDBE0E2EA93B8CBE89423F8E0E0E0935D
:100978001D020895A0918E01B0918F018091900180
:10098800909191010895E0938E01F0938F01609307
:100998009001709391010895E0911E02A6E2B0E0E3
:1009A800D1DFEE0FFF1FEA0FFB1F0895EA9394CBE8
:1009B800EA93B0DC662777270895E0936201F09305
:1009C800630160936401709365010895E093660183
:1009D800F093670160936801709369010895E0934B
:1009E8006A01F0936B0160936C0170936D01089537
:1009F800E0936E01F0936F01609370017093710141
:100A08000895E0937201F0937301609374017093F9
:100A180075010895A0919901B0919A010895AADFEE
:100A2800FF27662777270895662777270895E09395
:100A38009301F09394016093950170939601089542
:100A4800E0917E01F0917F010895EEDFBDD0DF01D6
:100A5800CB01E8E6F1E060E070E0DBD00895A0911A
:100A68006E01B0916F0180917001909171010895AC
:100A7800AF3FE3E0BE07E0E08E07E0E09E070895A1
:100A880099D0089582D0E2E2F1E060E070E0BCD055
:100A98000895A0917201B0917301809174019091B1
:100AA80075010895E8814EDFE456FE4F0895FE0172
:100AB8003396DF01EC910895ECE9F1E0FA93EA93BB
:100AC8000895FA93EA930895E0916001F091610125
:100AD8000895FE013396F5CF2BD0EECFEEE6F0E089
:100AE800F0DF35C0DBD0FE013596EBDFE8DEE4CF82
:100AF800EA83FB836C837D830895A885B9858A85FD
:100B08009B850895E887F9876A877B870895AE8172
:100B1800BF811196AE83BF8311970895EA81FB8147
:100B28006C817D81EACFAA81BB818C819D810895EA
:100B3800E991F991A991B991CD016D916623E9F7F0
:100B4800119761916D936623E1F7FC010895E9918E
:100B5800F991A991B991CD016D916623E9F71197A2
:100B680005900D920020E1F7FC010895A991B99133
:100B7800EE27FF276D91662311F03196FBCF08957C
:100B8800EA0FFB1F681F791F0895AE1BBF0B860B6A
:100B9800970B0895F09560957095E195FF4F6F4F0D
:100BA8007F4F0895EE230E2EEA2F19F0EE0F0A94C8
:100BB800E9F708956F2F660F660B762F0895EA17E9
:100BC800E1E009F0EE2708957A9F702D6B9F700D74
:100BD800F89F700DE99F700D6A9F602D710DFB9F46
:100BE800600D711DE89F600D711D8827FA9FF02D1B
:100BF800610D781FEB9FF00D611D781FEA9FE02DB6
:100C0800F10D681F781F089532D0DEDF0EF4C2DFC1
:100C180008953F934F935F93002411244427552749
:100C280030E2AA0FBB1F881F991F001C111C441F0C
:100C3800551F0E1A1F0A460B570B28F40E0E1F1EBF
:100C4800461F571F01C0A1603A9559F7FD01BC0125
:100C5800D001CA015F914F913F91089508D0D9DF23
:100C68000EF498DF0895D5DFFD01BC010895E894DE
:100C780077FF02C08FDF689497FF0BC00024A09510
:100C8800B095809590951196801D901D00F803945D
:100C980000FA08950590F491E02D08957A936A93E7
:100CA800FA93EA930895119602D0FE2F1197E199CD
:100CB800FECFFF93FFB7F894AEBBBFBBE09AEDB38E
:100CC800FFBFFF91089530976040704008951097D6
:100CD8008040904008951A930A93089519810881D5
:100CE8000895AC0FBD1F05900D928A95E1F7089500
:00000001FF
